:020000000F28C7
:10000800FE00030EF1000408F2000A08F300831250
:100018007F08F4007428A0288B0107308312990008
:10002800703083169F0004309100093083129F00BE
:10003800F9308316920005308312920093010C3038
:1000480095000430831685008312850103308316DA
:100058008700033083128700843083168100F601FD
:100068007D30F5007508F800F7010630831281002D
:100078008B168B173F28F930F5000000F50B412847
:100088004528000083129F1449289F184C284D28A2
:1000980049284E281E08F5007508F6000730760234
:1000A8000318572858285D280730F5007508F6000A
:1000B8005D288718602861286D2807186428652836
:1000C8006A28FF30F5007508F6006D28F6016D28DE
:1000D8006D287603FF3AFF3E93003F283F280F28FC
:1000E8000B1D7728782895280B11063081000130E0
:1000F800F802F808031D812882288A287D30F0003C
:100108007008F8000430F0007008F7007708031D45
:100118008E2892280130F70207169528071295288D
:1001280095287408FF0073088A0072088400710E0D
:100138008300FE0E7E0E0900F601F70183011028E8
:02400E00E1F3DC
:00000001FF
